:020000020000FC
:1000000014C00000000000000EC00BC036F07A954E
:1000100019F47EBD73BFA068189556E05EBDE894E4
:100020001895B3951895939518955FED5DBF52E0BF
:1000300051BB5FEF57BB5FEF58BB52BB54E359B99D
:1000400058E05AB955275BBD5AE65ABD78945CE230
:1000500058BB55E489D152E0052EEFD15CEB58BB7B
:100060005CE482D154E1052EE8D15AE258BB53E555
:100070007BD158E0E2D15BED58BB59E475D154E037
:10008000052EDBD15CE258BB55E46ED152E0052E63
:10009000D4D15CE458BB52E367D157E2052ECDD1F1
:1000A0005FEF58BB5AE060D15DE05ED150E859BFC8
:1000B000AA27BB2756E05EBDB031F1F755275EBDDC
:1000C00052E059BFA16034C0829BFECF839BFCCF1E
:1000D000849BFACF829B2CC0839B29C0849B01C048
:1000E000F9CF8FE09927849905C09F3FE1F78A9562
:1000F000C9F7E8CF55275EBD52E059BF55275DBD12
:100100005CBDBB2772E352E859BF689453E053BF0C
:10011000A7FFFECFAF7752E059BF7CB48DB49B2EC2
:10012000AA24CBD0A062E5D024D1AF7DCDCFA064EE
:1001300055275EBD52E059BF55275DBD5CBD72E3DA
:10014000689453E053BFA7FFFECFAF770CB41DB444
:100150000BD0A0FF05C05AE0052E6FD1AE7FB4CF03
:10016000C8D007D1AD7BB0CF802C912C52D0A6FD4A
:1001700007C05CEF852E53E0952EAA24BB2408C04F
:100180008090700090907100A0907200B090730009
:100190004FD0772450E2852E59E2952E54E3A52EB8
:1001A00050E8B52E5DEFC52E59E5D52E5AD0A0FDED
:1001B00027C0A6FF07C05CEF052E53E0152E2224B2
:1001C000332408C0009070001090710020907200DD
:1001D00030907300701881089208A30810F06DD059
:1001E0000895700C811C921CA31C0718180829087C
:1001F0003A08702C812C922CA32CA2605ED008951A
:10020000709270008092710090927200A0927300C0
:1002100008952224332480E11694079410F4280CC6
:10022000391C37942794179407948A95B9F7089541
:10023000442455246624772480E236942794179426
:10024000079420F4480C591C6A1C7B1C7794679413
:100250005794479437942794179407948A9589F76D
:100260000895FF240027112722273327442789E3F5
:10027000EE18771C881C991CAA1CBB1CCC1CDD1C0E
:100280008A9509F40895EE1CFF1C001F111F221F00
:10029000331F441FE018F108020913092409350926
:1002A000460948F4E00CF11C021D131D241D351DE8
:1002B000461D8894DECF0894DCCF88E1FF24EE242D
:1002C000DD240027770C881C991CDD1CEE1CFF1C0C
:1002D000001F8A9509F40895E1E1FF2752915D5FBF
:1002E00053FD50835081505D57FD5083ED30B1F781
:1002F000E9CF5CE4A6FD53E4A5FD56E435D050E219
:1003000033D0A1FF02C05DE22FD0002329F4FF20EB
:1003100051F4EE2079F415C0502F52955F7023D020
:10032000502F5F7020D05F2D52955F701CD05F2DD5
:100330005F7019D05E2D52955F7015D05E2D5F7085
:1003400012D0A6FD04C0A5FD02C05EE20DD05D2D59
:1003500052955F7008D05D2D5F7005D05AE004D0D3
:100360005DE002D0089550635CB95BB155FFFDCFED
:1003700008955CEBA6FD5CE3A5FD5DE258BB54E18E
:10038000A6FD5AE1A5FD52E1052E57D0A1FF05C0FB
:100390005FEE58BB53E7052E50D0002329F4FF2011
:1003A00061F4EE2099F41BC0502F52955F7038D045
:1003B0002BD0502F5F7034D027D05F2D52955F70B7
:1003C0002FD022D05F2D5F702BD01ED05E2D529586
:1003D0005F7026D019D05E2D5F7022D015D0A6FD9B
:1003E00007C0A5FD05C05FEE58BB5AE0052E25D01D
:1003F0005D2D52955F7014D007D05D2D5F7010D0C9
:1004000003D05FEF58BB0895F4E0E6E1E50F002468
:10041000F01DC89512C03F2F2723212030383C3EC5
:10042000F4E0E0E3E50F0024F01DC89508BA089554
:1004300018DB4C4A8B2AA85B080B55275DBD5CBDB9
:1004400050E459BF5BE05EBD88E0001C8A95E8F788
:10045000992750E45FBD001C18F09035F1F702C0F9
:10046000903FF1F750E05FBD99279035F1F78A95FD
:1004700079F777E099279035F1F77A95D9F70895CC
:00000001FF
